******************************************************************************
             TMS470 COFF Linker PC v4.1.2                      
******************************************************************************
>> Linked Thu May 03 11:05:19 2012

OUTPUT FILE NAME:   <./Debug/UCD3138_Lab_04.out>
ENTRY POINT SYMBOL: "_c_int00"  address: 00000c44


MEMORY CONFIGURATION

                  name            origin    length      used    attr    fill
         ----------------------  --------  ---------  --------  ----  --------
         VECS                    00000000   00000020  00000020  RWIX
         PFLASH                  00000020   00007f38  00000d5b  R  X
         DEVICEID                00007f58   00000020  00000000  R  X
         FIXTFA                  00007f78   00000004  00000000  R  X
         FIXCONST                00007f7c   00000080  00000000  R  X
         FLASHSUM                00007ffc   00000004  00000000  R  X
         ROM                     0000a020   00001d5e  00000000  RWIX
         SINE                    0000bd7e   00000282  00000000  RWIX
         DFLASH                  00018800   00000800  00000000  R  X
         TESTER                  00019000   0000001c  00000000  RW  
         RAM                     0001901c   00000e50  00000050  RW  
         STACKS                  00019e6c   00000190  00000000  RW  
         ROMLOCK                 00019ffc   00000004  00000000  RW  
         LOOP_MUX                00020000   00000078  00000078  RWIX
         FAULT_MUX               00030000   00000080  00000080  RWIX
         ADC                     00040000   00000098  00000098  RWIX
         DPWM3                   00050000   0000008c  0000008c  RWIX
         FILTER2                 00060000   00000064  00000064  RWIX
         DPWM2                   00070000   0000008c  0000008c  RWIX
         FE_CTRL2                00080000   00000044  00000044  RWIX
         FILTER1                 00090000   00000064  00000064  RWIX
         DPWM1                   000a0000   0000008c  0000008c  RWIX
         FE_CTRL1                000b0000   00000044  00000044  RWIX
         FILTER0                 000c0000   00000064  00000064  RWIX
         DPWM0                   000d0000   0000008c  0000008c  RWIX
         FE_CTRL0                000e0000   00000044  00000044  RWIX
         UART0                   fff7ec00   00000038  00000038  RWIX
         UART1                   fff7ed00   00000038  00000038  RWIX
         MISC_ANALOG             fff7f000   00000048  00000048  RWIX
         PMBUS                   fff7f600   00000024  00000024  RWIX
         GIO                     fff7fa00   00000040  00000040  RWIX
         TIMER                   fff7fd00   0000009c  0000009c  RWIX
         MMC                     fffffd00   0000003c  0000003c  RWIX
         DEC                     fffffe00   0000009c  0000009c  RWIX
         CIM                     ffffff20   00000018  00000018  RWIX
         SYS                     ffffffd0   00000030  00000030  RWIX


SECTION ALLOCATION MAP

 output                                  attributes/
section   page    origin      length       input sections
--------  ----  ----------  ----------   ----------------
Uart0RegsFile 
*          0    fff7ec00    00000038     UNINITIALIZED
                  fff7ec00    00000038     cyclone_global_variables_defs.obj (Uart0RegsFile)

Uart1RegsFile 
*          0    fff7ed00    00000038     UNINITIALIZED
                  fff7ed00    00000038     cyclone_global_variables_defs.obj (Uart1RegsFile)

MiscAnalogRegsFile 
*          0    fff7f000    00000048     UNINITIALIZED
                  fff7f000    00000048     cyclone_global_variables_defs.obj (MiscAnalogRegsFile)

PMBusRegsFile 
*          0    fff7f600    00000024     UNINITIALIZED
                  fff7f600    00000024     cyclone_global_variables_defs.obj (PMBusRegsFile)

GioRegsFile 
*          0    fff7fa00    00000040     UNINITIALIZED
                  fff7fa00    00000040     cyclone_global_variables_defs.obj (GioRegsFile)

TimerRegsFile 
*          0    fff7fd00    0000009c     UNINITIALIZED
                  fff7fd00    0000009c     cyclone_global_variables_defs.obj (TimerRegsFile)

MmcRegsFile 
*          0    fffffd00    0000003c     UNINITIALIZED
                  fffffd00    0000003c     cyclone_global_variables_defs.obj (MmcRegsFile)

DecRegsFile 
*          0    fffffe00    0000009c     UNINITIALIZED
                  fffffe00    0000009c     cyclone_global_variables_defs.obj (DecRegsFile)

CimRegsFile 
*          0    ffffff20    00000018     UNINITIALIZED
                  ffffff20    00000018     cyclone_global_variables_defs.obj (CimRegsFile)

SysRegsFile 
*          0    ffffffd0    00000030     UNINITIALIZED
                  ffffffd0    00000030     cyclone_global_variables_defs.obj (SysRegsFile)

//data     0    00000000    00000000     UNINITIALIZED

flash      0    00000000    00000000     UNINITIALIZED

.data      0    00000000    00000000     UNINITIALIZED

.vectors   0    00000000    00000020     
                  00000000    00000020     load.obj (.vectors)

.fiq       0    0000001c    00000000     UNINITIALIZED

.cinit     0    00000020    00000000     UNINITIALIZED

.text      0    00000020    00000c40     
                  00000020    000002d8     pmbus_handler.obj (.text)
                  000002f8    00000234     pmbus_manuf_specific_commands.obj (.text)
                  0000052c    00000218     interrupts.obj (.text)
                  00000744    00000168     main.obj (.text)
                  000008ac    00000134     pmbus.obj (.text)
                  000009e0    000000d8     load.obj (.text)
                  00000ab8    000000bc     pmbus_manuf_info_commands.obj (.text)
                  00000b74    0000008c     clear_program_flash.obj (.text)
                  00000c00    00000024     init_pmbus.obj (.text)
                  00000c24    00000020     rts32tiabi.lib : icall32.obj (.text)
                  00000c44    00000018     main.obj (.text:v$6)
                  00000c5c    00000004     standard_interrupt.obj (.text)

.const     0    00000c60    0000011b     
                  00000c60    000000b2     pmbus_manuf_specific_commands.obj (.const)
                  00000d12    00000002     --HOLE-- [fill = 0]
                  00000d14    00000067     pmbus_manuf_info_commands.obj (.const)

FixedDeviceID 
*          0    00007f58    00000000     UNINITIALIZED

FixedTfaStep 
*          0    00007f78    00000000     UNINITIALIZED

FixedConstants 
*          0    00007f7c    00000000     UNINITIALIZED

.flashi    0    00007ffc    00000000     UNINITIALIZED

.sine      0    0000bd7e    00000000     UNINITIALIZED

.dflash    0    00018800    00000000     UNINITIALIZED

.CONFIG    0    00018800    00000000     UNINITIALIZED

.CONFIG_B 
*          0    00018800    00000000     UNINITIALIZED

.PASSW     0    00018800    00000000     UNINITIALIZED

TesterVars 
*          0    00019000    00000000     UNINITIALIZED

.bss       0    0001901c    00000050     UNINITIALIZED
                  0001901c    00000050     main.obj (.bss)

.stack     0    00019e6c    00000000     UNINITIALIZED

.romlock   0    00019ffc    00000000     UNINITIALIZED

LoopMuxRegsFile 
*          0    00020000    00000078     UNINITIALIZED
                  00020000    00000078     cyclone_global_variables_defs.obj (LoopMuxRegsFile)

FaultMuxRegsFile 
*          0    00030000    00000080     UNINITIALIZED
                  00030000    00000080     cyclone_global_variables_defs.obj (FaultMuxRegsFile)

AdcRegsFile 
*          0    00040000    00000098     UNINITIALIZED
                  00040000    00000098     cyclone_global_variables_defs.obj (AdcRegsFile)

Dpwm3RegsFile 
*          0    00050000    0000008c     UNINITIALIZED
                  00050000    0000008c     cyclone_global_variables_defs.obj (Dpwm3RegsFile)

Filter2RegsFile 
*          0    00060000    00000064     UNINITIALIZED
                  00060000    00000064     cyclone_global_variables_defs.obj (Filter2RegsFile)

Dpwm2RegsFile 
*          0    00070000    0000008c     UNINITIALIZED
                  00070000    0000008c     cyclone_global_variables_defs.obj (Dpwm2RegsFile)

FeCtrl2RegsFile 
*          0    00080000    00000044     UNINITIALIZED
                  00080000    00000044     cyclone_global_variables_defs.obj (FeCtrl2RegsFile)

Filter1RegsFile 
*          0    00090000    00000064     UNINITIALIZED
                  00090000    00000064     cyclone_global_variables_defs.obj (Filter1RegsFile)

Dpwm1RegsFile 
*          0    000a0000    0000008c     UNINITIALIZED
                  000a0000    0000008c     cyclone_global_variables_defs.obj (Dpwm1RegsFile)

FeCtrl1RegsFile 
*          0    000b0000    00000044     UNINITIALIZED
                  000b0000    00000044     cyclone_global_variables_defs.obj (FeCtrl1RegsFile)

Filter0RegsFile 
*          0    000c0000    00000064     UNINITIALIZED
                  000c0000    00000064     cyclone_global_variables_defs.obj (Filter0RegsFile)

Dpwm0RegsFile 
*          0    000d0000    0000008c     UNINITIALIZED
                  000d0000    0000008c     cyclone_global_variables_defs.obj (Dpwm0RegsFile)

FeCtrl0RegsFile 
*          0    000e0000    00000044     UNINITIALIZED
                  000e0000    00000044     cyclone_global_variables_defs.obj (FeCtrl0RegsFile)


GLOBAL SYMBOLS: SORTED ALPHABETICALLY BY Name 

address    name
--------   ----
00000878   $c_int00
0000080e   $global_enable
00000744   $init_dpwm0
00000790   $init_filter0
0000081a   $init_front_end0
000007fa   $init_loop_mux
00000c00   $init_pmbus
00000832   $main
00000020   $pmbus_handler
000000fa   $pmbus_idle_handler
00000b20   $pmbus_mfr_date_handler
00000b12   $pmbus_mfr_id_handler
00000b2e   $pmbus_mfr_location_handler
00000af6   $pmbus_mfr_model_handler
00000b04   $pmbus_mfr_revision_handler
00000b3c   $pmbus_mfr_serial_handler
000001de   $pmbus_read_block_handler
0000031c   $pmbus_read_cmd_dcdc_nonpaged
000002f8   $pmbus_read_cmd_dcdc_paged
00000ada   $pmbus_read_device_id
000008f8   $pmbus_read_message
000008ac   $pmbus_read_one_byte_handler
00000392   $pmbus_read_parm_info
00000494   $pmbus_read_parm_value
00000ae8   $pmbus_read_setup_id
000008ba   $pmbus_read_two_byte_handler
000002aa   $pmbus_read_wait_for_eom_handler
00000058   $pmbus_write_block_handler
000008cc   $pmbus_write_message
00000348   $pmbus_write_parm_info
000003be   $pmbus_write_parm_value
00000340   $pmbus_write_rom_mode
00000ab8   $send_string
0001901c   .bss
00000000   .data
00000020   .text
00000c24   IND_CALL
00019054   _A_string
00040000   _AdcRegs
ffffff20   _CimRegs
fffffe00   _DecRegs
000d0000   _Dpwm0Regs
000a0000   _Dpwm1Regs
00070000   _Dpwm2Regs
00050000   _Dpwm3Regs
00030000   _FaultMuxRegs
000e0000   _FeCtrl0Regs
000b0000   _FeCtrl1Regs
00080000   _FeCtrl2Regs
000c0000   _Filter0Regs
00090000   _Filter1Regs
00060000   _Filter2Regs
fff7fa00   _GioRegs
00020000   _LoopMuxRegs
fff7f000   _MiscAnalogRegs
fffffd00   _MmcRegs
fff7f600   _PMBusRegs
00019fec   _StackABORT_
00019f94   _StackFIQ_
00019fe8   _StackIRQ_
00019ffc   _StackSUPER_
00019ff0   _StackUND_
00019f24   _StackUSER_
ffffffd0   _SysRegs
fff7fd00   _TimerRegs
fff7ec00   _Uart0Regs
fff7ed00   _Uart1Regs
ffffffff   ___binit__
0001901c   ___bss__
ffffffff   ___c_args__
ffffffff   ___cinit__
00000000   ___data__
00000000   ___edata__
0001906c   ___end__
00000c60   ___etext__
ffffffff   ___pinit__
00000020   ___text__
0000071c   _abort_data_fetch_exception
00000718   _abort_prefetch_exception
00000c44   _c_int00
00000b74   _clear_program_flash
00000c80   _cmd_dcdc_nonpaged
00000c60   _cmd_dcdc_paged
00000d5c   _device_id_string
00000720   _fast_interrupt
00000d40   _mfr_date
00000d24   _mfr_id
00000d48   _mfr_location
00000d28   _mfr_model
00000d3c   _mfr_revision
00000d54   _mfr_serial
00019020   _parm_count
0001901c   _parm_index
00000cec   _parm_mem_length
00000ca0   _parm_mem_start
0001901e   _parm_offset
00019021   _parm_size
00019024   _pmbus_buffer
0001904e   _pmbus_buffer_position
0001904d   _pmbus_number_of_bytes
0001904c   _pmbus_state
00019050   _pmbus_status_half_word_0_value
00019052   _pmbus_status_half_word_0_value_ored
00019068   _ram_eadcdac
00000d14   _setup_id
00000530   _software_interrupt
00000c5c   _standard_interrupt
0000052c   _undefined_instruction_exception
00000b94   _zero_out_integrity_word
ffffffff   binit
ffffffff   cinit
00000000   edata
0001906c   end
00000c60   etext
ffffffff   pinit
ffffa4dc   rom_main


GLOBAL SYMBOLS: SORTED BY Symbol Address 

address    name
--------   ----
00000000   edata
00000000   .data
00000000   ___edata__
00000000   ___data__
00000020   .text
00000020   $pmbus_handler
00000020   ___text__
00000058   $pmbus_write_block_handler
000000fa   $pmbus_idle_handler
000001de   $pmbus_read_block_handler
000002aa   $pmbus_read_wait_for_eom_handler
000002f8   $pmbus_read_cmd_dcdc_paged
0000031c   $pmbus_read_cmd_dcdc_nonpaged
00000340   $pmbus_write_rom_mode
00000348   $pmbus_write_parm_info
00000392   $pmbus_read_parm_info
000003be   $pmbus_write_parm_value
00000494   $pmbus_read_parm_value
0000052c   _undefined_instruction_exception
00000530   _software_interrupt
00000718   _abort_prefetch_exception
0000071c   _abort_data_fetch_exception
00000720   _fast_interrupt
00000744   $init_dpwm0
00000790   $init_filter0
000007fa   $init_loop_mux
0000080e   $global_enable
0000081a   $init_front_end0
00000832   $main
00000878   $c_int00
000008ac   $pmbus_read_one_byte_handler
000008ba   $pmbus_read_two_byte_handler
000008cc   $pmbus_write_message
000008f8   $pmbus_read_message
00000ab8   $send_string
00000ada   $pmbus_read_device_id
00000ae8   $pmbus_read_setup_id
00000af6   $pmbus_mfr_model_handler
00000b04   $pmbus_mfr_revision_handler
00000b12   $pmbus_mfr_id_handler
00000b20   $pmbus_mfr_date_handler
00000b2e   $pmbus_mfr_location_handler
00000b3c   $pmbus_mfr_serial_handler
00000b74   _clear_program_flash
00000b94   _zero_out_integrity_word
00000c00   $init_pmbus
00000c24   IND_CALL
00000c44   _c_int00
00000c5c   _standard_interrupt
00000c60   _cmd_dcdc_paged
00000c60   etext
00000c60   ___etext__
00000c80   _cmd_dcdc_nonpaged
00000ca0   _parm_mem_start
00000cec   _parm_mem_length
00000d14   _setup_id
00000d24   _mfr_id
00000d28   _mfr_model
00000d3c   _mfr_revision
00000d40   _mfr_date
00000d48   _mfr_location
00000d54   _mfr_serial
00000d5c   _device_id_string
0001901c   .bss
0001901c   ___bss__
0001901c   _parm_index
0001901e   _parm_offset
00019020   _parm_count
00019021   _parm_size
00019024   _pmbus_buffer
0001904c   _pmbus_state
0001904d   _pmbus_number_of_bytes
0001904e   _pmbus_buffer_position
00019050   _pmbus_status_half_word_0_value
00019052   _pmbus_status_half_word_0_value_ored
00019054   _A_string
00019068   _ram_eadcdac
0001906c   ___end__
0001906c   end
00019f24   _StackUSER_
00019f94   _StackFIQ_
00019fe8   _StackIRQ_
00019fec   _StackABORT_
00019ff0   _StackUND_
00019ffc   _StackSUPER_
00020000   _LoopMuxRegs
00030000   _FaultMuxRegs
00040000   _AdcRegs
00050000   _Dpwm3Regs
00060000   _Filter2Regs
00070000   _Dpwm2Regs
00080000   _FeCtrl2Regs
00090000   _Filter1Regs
000a0000   _Dpwm1Regs
000b0000   _FeCtrl1Regs
000c0000   _Filter0Regs
000d0000   _Dpwm0Regs
000e0000   _FeCtrl0Regs
fff7ec00   _Uart0Regs
fff7ed00   _Uart1Regs
fff7f000   _MiscAnalogRegs
fff7f600   _PMBusRegs
fff7fa00   _GioRegs
fff7fd00   _TimerRegs
ffffa4dc   rom_main
fffffd00   _MmcRegs
fffffe00   _DecRegs
ffffff20   _CimRegs
ffffffd0   _SysRegs
ffffffff   pinit
ffffffff   ___pinit__
ffffffff   ___c_args__
ffffffff   ___binit__
ffffffff   ___cinit__
ffffffff   cinit
ffffffff   binit

[116 symbols]
